:020000040000FA
:1000000048140020150200001D0200001F0200001D
:100010002102000023020000250200000000000071
:1000200000000000000000000000000027020000A7
:1000300029020000000000002B0200002D02000039
:100040002F020000A5020000310500002F02000071
:100050002F020000000000002F020000000000003E
:100060002F0200002F0200002F0200002F020000CC
:100070002F0200002F0200002F0200002F020000BC
:100080002F0200002F0200002F0200002F020000AC
:10009000010300002F0200002F0200002F020000C9
:1000A0002F0200002F0200002F02000000000000BD
:1000B0000000000000000000000000000000000040
:1000C0000000000000000000000000000000000030
:1000D0000000000000000000000000002F020000EF
:1000E0000000000000000000000000000000000010
:1000F0000000000000000000000000000000000000
:1001000000000000000000000000000000000000EF
:1001100000000000000000000000000000000000DF
:1001200000000000000000000000000000000000CF
:1001300000000000000000000000000000000000BF
:1001400000000000000000000000000000000000AF
:10015000000000000000000000000000000000009F
:10016000000000000000000000000000000000008F
:10017000000000000000000000000000000000007F
:10018000000000000000000000000000000000006F
:10019000000000000000000000000000000000005F
:1001A000000000000000000000000000000000004F
:1001B000000000000000000000000000000000003F
:1001C000000000000000000000000000000000002F
:1001D000000000000000000000000000000000001F
:1001E000000000000000000000000000000000000F
:1001F00000000000000000000000000000000000FF
:10020000DFF80CD000F03CF800480047110800006F
:10021000481400200648804706480047FEE7FEE7EE
:10022000FEE7FEE7FEE7FEE7FEE7FEE7FEE7FEE7A6
:10023000590300000102000040EA01039B0703D0BC
:1002400009E008C9121F08C0042AFAD203E011F815
:10025000013B00F8013B521EF9D27047D2B201E0D7
:1002600000F8012B491EFBD270470022F6E710B5BB
:1002700013460A4604461946FFF7F0FF204610BD14
:10028000064C074D06E0E06840F0010394E80700E3
:1002900098471034AC42F6D3FFF7B6FFD8120000EF
:1002A000F812000070B5144CD4F80001002628B1F3
:1002B000D4F80403C00701D0C4F80061D4F80C01DD
:1002C0000E4D40B1D4F80403000704D5C4F80C6106
:1002D000286900B18047D4F8100100280BD0D4F869
:1002E0000403C00607D5C4F81061E868002802D0EE
:1002F000BDE87040004770BD001000403000002095
:100300007CB5144C606A01902078002821D001202F
:1003100000F021F9656800266660012000F02CF9E4
:10032000E169002915D0E80703D08DF80060684620
:100330008847A80705D501208DF80000E1696846C7
:100340008847680705D502208DF80000E1696846F6
:1003500088477CBD30000020F0B54FF08051684FD9
:10036000D1F83001674E421C09D0D1F83441034620
:10037000012500220D2B07D0102B05D00FE032787D
:100380003B78C2F30314F3E70CB1012C07D14FF013
:100390008043C3F80C21C3F810215B4B1A60431C47
:1003A00007D0D1F8344103460D2B07D0102B05D0D0
:1003B0005DE034783B78C4F30314F5E70CB1012C0D
:1003C00055D1524B1B68524C2360504B1B1D1B6870
:1003D000241D23604D4B08331B68241D23604B4BA9
:1003E0000C331B68241D2360484B10331B68241DED
:1003F0002360464B14331B68241D2360434B183382
:100400001B68434C20342360404B1C331B68241D65
:1004100023603E4B20331B68241D23603B4B243359
:100420001B68241D2360394B28331B68241D23605F
:10043000364B2C331B68241D2360344B30331B6830
:10044000334C40342360314B34331B68241D23600C
:100450002E4B38331B68241D23602C4B3C331B6808
:10046000241D2360294B40331B68241D2360431C3B
:1004700006D0D1F834110D2807D0102805D00EE091
:1004800031783878C1F30311F5E709B1012906D1B4
:1004900020480168C90702D06FF0010101604FF0E8
:1004A0001021D1F80002002803DBD1F80402002853
:1004B00021DA194C256019480368002BFCD012235F
:1004C000C1F800320568002DFCD0C1F80432016883
:1004D0000029FCD0226001680029FCD0BFF34F8FB7
:1004E0000F4801680F4A01F4E06111430160BFF356
:1004F0004F8F00BFFDE70D490B480860F0BD0000BD
:10050000E00F00F0E80F00F0380500400404001090
:1005100020C500400004004004E5014000E4014023
:100520000CED00E00400FA050090D00378000020F4
:10053000014800680047000028000020002809DB6F
:1005400000F01F02012191404009800000F1E020ED
:10055000C0F88012704700280DDB00F01F02012157
:1005600091404009800000F1E020C0F88011BFF305
:100570004F8FBFF36F8F7047002809DB00F01F0219
:10058000012191404009800000F1E020C0F80011F5
:100590007047002809DB00F01F020121914040094B
:1005A000800000F1E020C0F8001270474907090EF2
:1005B000002804DB00F1E02080F80014704700F010
:1005C0000F0000F1E02080F8141D704702E008C819
:1005D000121F08C1002AFAD170477047002001E0BD
:1005E00001C1121F002AFBD17047006890FAA0F0E9
:1005F00000BA00BA7047000072B609480068C00728
:1006000000D000BEBFF34F8F0548E4380168054AAB
:1006100001F4E06111430160BFF34F8F00BFFDE7BC
:10062000F0ED00E00400FA050EB500210091CDE9DF
:1006300001106A4644F20100FFF7DEFF0EBD000024
:100640002DE9FC410646C0074FF000050ED0104FC3
:1006500000240122385D009500231146019500F029
:1006600059FB641C042CF4D300F01CF8B0070DD522
:10067000074E0024361D0022305D032300951146ED
:10068000019500F047FB641C042CF4D3BDE8FC8109
:10069000D01200000249085C012100F058BB0000A4
:1006A000D012000010B500242046FFF7F3FF641CB1
:1006B000042CF9D310BD006890FAA0F000BA70477E
:1006C0004FF080400021C0F800110121C0F8001057
:1006D000D0F800110029FBD07047000000B51BA026
:1006E0008BB0006808901AA01AA100680990D1E99F
:1006F0000001CDE90601182218496846FFF79CFD64
:1007000001208DF800008DF80800154801900020A8
:100710008DF801004FF416718DF81400ADF80C102F
:10072000684600F017F900280DD108A800F0DCF9A0
:10073000002808D109A800F0E9F9002803D1082110
:1007400006A800F0F5F90BB000BD0000E7E7E7E709
:10075000C2C2C2C2E7C2C3C4C5C6C7C8B81200007D
:10076000F908000030B408200F214FF0A043032205
:1007700003EB8004C4F80027401C8842F8D930BC41
:100780000120FFF75DBF000070B500F0E3FB1E49DC
:100790000020A1F5947300BF00EB800202EB401231
:1007A0001A4441F82020401C0828F5DB1649002097
:1007B0002C3101F5947200BF00EB800404EB40146F
:1007C0000C4442F82040401C0828F5DB00200F4A6A
:1007D0004FEA000100EB800404EB4014E51800EB45
:1007E0004004401C42F8245002EB84040828217184
:1007F000A160EFDB054A002012F1600242F82010F0
:10080000401C0828FADB70BDE4010020A80300208A
:10081000FFF7A8FFFFF754FFFFF760FF08B1FFF7EE
:1008200003FF214C214D224E0027E7701E4800F0A7
:10083000D9F9A0BBA079410703D000F00700042834
:1008400001D9012100E000210D2000F075FAA07906
:1008500000F00700012801D9052801D9012100E095
:1008600000210E2000F068FAA07900F007000228AD
:1008700001D9062801D9012100E000210F2000F054
:100880005BFAA07900F00700032801D8012100E0FD
:100890000021102000F050FAA079401CA071691CC2
:1008A00030468847C1E7000000000020B012000079
:1008B00000D4300070B50C494FF4705008600B4CF8
:1008C00000256570257000F045FB20210848FFF7E2
:1008D000CCFCE56214202563FFF73DFE05490320AB
:1008E000C1F80002002070BD08F501403000002072
:1008F000280400200010004010B50078002808D01F
:10090000012807D0022804D1054800F0A9F80028E2
:10091000FAD010BD00F006F8BDE8104000F04EB966
:100920007C000020094810B5007860B10120FFF775
:1009300012FE074800218162016241620120FFF737
:100940001BFE002010BD082010BD0000300000205C
:10095000E401002070B5050065D0354C207818B151
:10096000FFF7A8FF00285DD16868E06118222946DA
:100970003048FFF761FC0025656020212E48FFF715
:1009800074FCE562256300F015FCE8B32B494FF0D9
:10099000E7300860091D4FF043300860091D284802
:1009A0000860091D27480860FFF7EEFE264904206D
:1009B0000860254808380560244840F20221C0F844
:1009C0000012244A22491160111D08602048001DB0
:1009D000091D08601D481030091D0860091D1E48CA
:1009E00008601B48F038091D08601B48001D091DE0
:1009F0000860091D194808600E4E707C00F0070160
:100A00000120FFF7D3FD00E00FE0B07C00F007010C
:100A10001420FFF7CBFD1420FFF7AEFD6570012019
:100A20002070002070BD0E2070BD072070BD00003A
:100A300030000020A4000020280400201C150040E5
:100A4000E743C323A363E31310A5004000A00040C5
:100A50000011004060F5014040A10040001000403E
:100A600070B505461E48007880B385B31D4CA06A5A
:100A700070B30120FFF76FFD606A54F820100A7808
:100A80002A7054F820104978697054F82010897839
:100A9000A97054F820100979297154F82010C978E8
:100AA000E97054F82010681D491DFFF7C5FB606A06
:100AB000401C6062082801D300206062A06A401ECA
:100AC000A0620120FFF758FD002070BD01E002E0A8
:100AD00003E00820F9E70E20F7E70520F5E700001E
:100AE0003000002038030020074910B54A780AB1C9
:100AF000112010BD30B100684863012000F00EFBEA
:100B0000002010BD0E2010BD30000020074910B598
:100B10004A780AB1112010BD30B100688863022004
:100B200000F0FCFA002010BD0E2010BD30000020A7
:100B300010B50C460F49497809B1112010BD18B104
:100B4000082C03D9072010BD0E2010BD014609480E
:100B500022463C30FFF770FB0648C4F108023430EF
:100B6000FF210474D1408174042000F0D7FA0020E2
:100B700010BD0000300000200E4810B50078A0B174
:100B80000D4CA06A98B10120FFF7E5FCA06A401E59
:100B9000A062606A401C6062082801D30020606285
:100BA0000120FFF7E9FC002010BD082010BD4FF424
:100BB000807010BD30000020E4010020074810B50F
:100BC000407808B1112010BD0548806A18B100F0C6
:100BD0001BFA002010BD4FF4807010BD30000020C3
:100BE000E40100202DE9F047DFF818A106469AF845
:100BF000000040B156B1307868B120280BD8424F80
:100C0000397829B109E00820BDE8F0870E20FBE71C
:100C1000F97C884201D90920F6E73C4CA06A0828F3
:100C200001D30420F0E77078082801D30720EBE710
:100C30000120FFF790FCDFF8CC8078784FF00009B6
:100C400008F12C0860B13249002000BF00EB4002DF
:100C500001EB82021279EAB1401C0828F6DB42E07F
:100C6000206A2522314654F82000FFF7E5FA727811
:100C700018F80210491C01F0030108F80210206A5C
:100C800054F82020401C08281171206228D3C4F891
:100C9000209025E000EB400011EB800523D00120DF
:100CA0002871C5F80890252231462868FFF7C4FA54
:100CB000727818F80210491C01F0030108F80210BC
:100CC0002868134A01717178603252F8210018B90E
:100CD00042F8215004E0084681680029FBD1856074
:100CE000A06A401CA0620120FFF746FC787830B96A
:100CF000387C20B99AF8010008B900F085F9002085
:100D000082E7000030000020A4000020E401002061
:100D1000A803002070B541EA4201DDE904564FF016
:100D2000A04441EA830141EA052104EB800041EA45
:100D30000641C0F8001770BD01224FF0A043824069
:100D400011B1C3F808257047C3F80C25704701227C
:100D50004FF0A043824011B1C3F808257047C3F893
:100D60000C25704770B5164CA068164AC2F80002F0
:100D7000A06A15490860154B091D988982380860DA
:100D80001348012140F80C1F0021C0F83411C0F8AD
:100D90003811104D4FF4E050286050142D1D28607C
:100DA000C2F80C11187810B96169002088470B4906
:100DB000094808600A48E0600320607070BD0000C8
:100DC000300000200010004040A50040A40000209A
:100DD00000A0004004F501408603002004150040F7
:100DE000210E000010B50C4C606840F001006060FE
:100DF000FFF7C2FE0948806A30B11420FFF7C9FB33
:100E0000BDE8104000F000B900206070BDE810405F
:100E10001420FFF7BEBB000030000020E4010020DA
:100E20002DE9F047414A4FF4E05010604049D1F8B5
:100E30000C31DFF8009100273F4CB9F80E004E143A
:100E4000DFF8F8800125E3B33D4B1B68CBB3256188
:100E50001660D8F8041041F00101C8F80410D8F861
:100E60002010401A401CC8F82400FFF785FE99F8AE
:100E7000000088B109F2E220017869B140784108A8
:100E800030480068C0B200F073F828B1D8F8040008
:100E900040F00400C8F804002B48806A50B199F86B
:100EA0001000012806D01420FFF773FBBDE8F047BF
:100EB00000F0AAB888F80170BDE8F0471420FFF7E9
:100EC00068BBD8F820C0BCF1010CC8F820C00BD218
:100ED00025611660401CC8F82400D8F8040040F0D2
:100EE0000200C8F80400E5E7D8F808000F4640F013
:100EF0000802C1F80022D8F81800D8F814100078B9
:100F0000884710481149283801601148C8F80C007A
:100F1000022088F8010025600448001F0660D4F80C
:100F20004401002800D03D60BDE8F08708F501408D
:100F300000100040A400002000A00040300000206D
:100F4000001400402C150040E40100206403002040
:100F5000650D00000549002008624862886201F5BD
:100F6000AA7108624862886270470000E4010020AC
:100F70002DE9F041224C07468846A06A08283DD258
:100F8000A4F5257120460A780026006A01F2E225C0
:100F9000012A03D04A7842B1C97C02E0297820298D
:100FA0002CD854F82020117002E054F820100E7054
:100FB00054F82000A91C10F8052BFFF73DF9206A12
:100FC00054F820104F700F49096854F82020917090
:100FD00054F8202082F80480697854F8202041F3E6
:100FE0000001491C401CD1702062082800D32662F1
:100FF000A06A401CA0620120BDE8F0810020FBE750
:1010000038030020481500402DE9F05F3D4C4FF0BB
:101010000108C4F824803C48DFF8F0A0A0F5A077D0
:10102000416A3B4D4FF0000B50F82110A161387818
:1010300007F5307610B1012843D10DE008786169D9
:101040008847A1690879307086F801B011F8052B3E
:10105000B01CFFF7F1F818E0C87820B3387D10B362
:10106000002081460878307008794006000E7070C4
:10107000CA78D2B100221043707011F8052BB01C51
:10108000FFF7DAF8B9F1000F11D0A06840F00800BE
:10109000C5F800021120C5F80403F8892062022077
:1010A000C4F80CA00CE00120DBE70122E3E7A06814
:1010B000C5F800021020C5F804031648E060404659
:1010C0006070A069144A417811604078444608FA7B
:1010D00000F0111D08600B480F4934302439C07CE2
:1010E0000860081F06600120FFF728FA0120FFF7BB
:1010F00043FAC5F804B1C5F808B1C5F810B12C60C1
:10110000BDE8F09F30000020E4010020650D0000E4
:1011100000100040E50D00002C15004010B50446FD
:10112000C00704D00F48FFF760FA0F490860A00716
:1011300006D50C48001DFFF758FA0B49091D086039
:1011400060070DD507480830FFF7B5FA06490831A2
:10115000086004480C30FFF7AEFA03490C31086010
:1011600010BD0000640000201C1500400E490F480F
:101170000A7A02600E48492352B1012A05D0032A97
:1011800006D0042A01D0002070473022826200E09D
:1011900083628B89826A3E32934202D2806A3E30F9
:1011A0008881012070470000A40000201015004035
:1011B0003000002070B500F03FF8FFF7D7FF184966
:1011C000184A0B787BB1012B0BD000230340164843
:1011D0004D7A041FB5B1012D0ED0022D07D0002489
:1011E00017E0124B00E0124B53610123EEE74FF67C
:1011F000FF7606600F4803E0FF26066040F2071006
:10120000206002E000260660266007480838056076
:101210000124C87C51691C408847204670BD0000ED
:10122000A4000020300000203C150040791200008E
:101230004D1200002110010002480349807A086025
:1012400070470000A40000200C150040084A074920
:1012500011600849497C491E090441EA0021014303
:1012600041F08070111D086070470000000101000E
:10127000141500406400002007490648086007482C
:101280000749407C401E41EA00400349091D0860AF
:1012900070470000060003001415004064000020A1
:1012A000200000010000000000000000000000001D
:1012B0000338FDD870470000010000000000000066
:1012C00001020000FA0003000001022000000000FB
:1012D0000D0E0F100B0C1819F81200000000002062
:1012E0007C000000CC050000741300007C0000208E
:1012F000CC130000DC050000080000000001000025
:1013000000110000000000000000000000000000CC
:1013100000000000000000000000000000000000CD
:1013200000000000000000000000000000000000BD
:101330001301000000000000000000000000000099
:10134000000000000000000000000000000000009D
:10135000000000000000000000000000E7E7E7E7F1
:10136000C2C2C2C2E7C2C3C4C5C6C7C80805FF021D
:041370000090D00316
:0400000500000201F4
:00000001FF
